:030000000212A742
:03000B000200C12F
:03002B000203EBE2
:03005B000205B8E3
:030073000205AED5
:1000800002030406080C10182030406080020304AC
:1000900006080C101820304080FF0406080C1018C9
:1000A0002030406080A0C000000001010003020277
:1000B000010D0D040206020D0505050D06030502DE
:1000C00002C2AFC0D0C0E0205A0D302F02E473301E
:1000D000600280F90203D7306306C283C294C295DE
:1000E00085258AC25AE525F4700221CA056130606F
:1000F00013206A19758B00D0E0D0D0C283C294C29D
:1001000095D2AF32C283C294C2950201BAD26EC2F6
:100110006FE565601CC3E5611495654014C26ED23D
:100120006FC3E561956450030201BA756100020175
:10013000BA206C14C283C294C2957408D5E0FDD273
:1001400080D282D2970201BAD26FC283C294C29582
:10015000E53D20E23420E1127408D5E0FD2075026F
:10016000D297307502D2800201BA20E0127408D50D
:10017000E0FD207502D297307502D2800201BA7478
:1001800008D5E0FDD2820201BA20E11F20E00A7406
:1001900008D5E0FDD2820201BA7408D5E0FD2075D1
:1001A00002D280307502D2970201BA7408D5E0FD00
:1001B000207502D280307502D297758B00D0E0D0C6
:1001C000D0C283C294C295D2AF32D0E0D0D0D2AFE9
:1001D0003261D7E525600A207502D283307502D2DC
:1001E00095C29461D7E5256002D294207502C2952C
:1001F000307502C28361D7E525600A207502D29569
:10020000307502D283207502C283307502C29561B7
:10021000D7207502C280307502C297E525600A209A
:100220007502D283307502D295207502C29730755F
:1002300002C280C29461D7207502C280307502C2AA
:1002400097207502C297307502C2807406D5E0FD12
:10025000E525600A207502D283307502D295C294DA
:1002600061D7207502C280307502C297E525600A09
:10027000207502D283307502D295C282C29461D7B2
:10028000207502C280307502C297C2827406D5E022
:10029000FDE525600A207502D283307502D295C231
:1002A0009461D7C282E5256002D294207502C28093
:1002B000307502C297207502C295307502C2836103
:1002C000D7C282207502C280307502C2977406D5EB
:1002D000E0FDE5256002D294207502C295307502DA
:1002E000C28361D7C282E5256002D294207502C222
:1002F00097307502C280207502C295307502C283A4
:1003000061D7C282207502C297307502C28074061E
:10031000D5E0FDE5256002D294207502C2953075C6
:1003200002C28361D7207502C297307502C280E590
:1003300025600A207502D295307502D283C28220D0
:100340007502C283307502C29561D7207502C297CB
:10035000307502C280C2827406D5E0FDE525600AD0
:10036000207502D295307502D283207502C2833087
:100370007502C29561D7207502C297307502C2809E
:10038000E525600A207502D295307502D28320756A
:1003900002C280307502C297207502C28330750296
:1003A000C29561D7207502C297307502C280207550
:1003B00002C280307502C2977406D5E0FDE5256063
:1003C0000A207502D295307502D283207502C2834D
:1003D000307502C29561D7E525F4F58A758B0075F5
:1003E0006000D25AD0E0D0D0D2AF32C2AFC0D0C0BD
:1003F000E0D2D3C2CEE528600A741F552E6049159D
:1004000028814878007900E580307601F430E502F3
:1004100078FF53DACF20760343DA2030760343DACD
:1004200010C2D8C269E580307601F430E50279FF68
:10043000C3E89970CE305903752840741F552E605B
:10044000037528408858D268E52960041529815B26
:10045000741F552E600543DA01C2D820680281E07E
:10046000E558F8C268741F552E60367982B704319A
:0F047000C3E894F0400374F0F8E8C4540F28F880
:10047F007984B7030281A1C313C313872120080214
:10048F00C313200A06C3C898F881A128F850037433
:10049F00FFF8C3E8955F5003E55FF8E52C5406704D
:1004AF0030882230630AC3E522955C4003855C22C5
:1004BF007882B6041CC3E5229524401278A096409A
:1004CF000DE52426F52450097524FF0204E085224A
:1004DF002420CF09D0E0D0D0C2D3D2AF32C2CF7850
:1004EF0001E5286008741F552E70021528C3E558C2
:1004FF0094014005755B00A10FE55B046002055B8D
:10050F007982B7020EE548601EC3E5229432401788
:10051F008547227982B7030FE548600BC3E5229424
:10052F00324004798E8722C3E52395226008400468
:10053F001523A1450523D8C80562E562700215622F
:10054F00D563537563017803C3E562941E4047C3B7
:10055F00E562946450087801756303020579C3E579
:10056F0062949650057801756301C3E55D9524404B
:10057F0018E548701485245DE56204600375621EFA
:10058F0075630175233C0205A5C3E55D285005750C
:10059F005DFFA1A5F55DD0E0D0D0C2D3D2AF32C2FE
:1005AF00AF53917FC258D2AF32C2AFC0D0C0E0C0FC
:1005BF00F0D2D3A8FBA9FCC2D8306902C11B53DA11
:1005CF00CF20760343DA1030760343DA20D269E581
:1005DF0080307601F420E502A1EF88268927E1BB60
:1005EF0053DACF20760343DA2030760343DA10C292
:1005FF00D8C269741F552E7002E1A17800E58030D2
:10060F007601F430E502E1A18858E1A153DACF2059
:10061F00760343DA2030760343DA10C26920590299
:10062F00C1D553DACF20760343DA1030760343DA9D
:10063F0020C2D8D26988538954C3E89551F8E995F7
:10064F0052F9E4FB7AFAC3E894C8E994005008E43D
:10065F00D2E4FB7A0AC1A8C3E89468E99401500870
:10066F00E4D2E3FB7A0FC1A8C3E894D0E994025017
:10067F0008E4D2E2FB7A1EC1A8C3E894A0E994056E
:10068F005008E4D2E1FB7A3CC1A8C3E89498E994FE
:10069F00085006E4D2E0FB7A78C3E89555FCE9955B
:1006AF0056FD30E708ECF42401FCEDF4FD7557001E
:1006BF007008C3EC9A500375570188558956A85393
:1006CF00A95488518952C3E89526F8E99527F9303E
:1006DF007402E174307302E174307202E16DE9C3A8
:1006EF0013F9E813F8307102E16DE9C313F9E81358
:1006FF00F8307002E16DE9C313FDE813FC205918BF
:10070F00C3EC941CED940240030207A1ED7009C3E2
:10071F00EC94C850030207BB74002077037896E669
:10072F0024FAFEE43400FFC3EC9EFCED9FFD50065F
:10073F0078007900E174C3EC94FFED9400400678E3
:10074F00FF7900E174EC856CF0A4C5F0A2F733F8E3
:10075F007900400302079078FF7900020790E9C300
:10076F0013F9E813F830740EE9600278FFC3E81349
:10077F0038F8E43400F9C3E894FFE99400400278B4
:10078F00FF8858D268205902E1A1741FF4552E4BEF
:10079F00F52E752840741F552E700375280A305991
:1007AF0002E1BB741F552E600353DAFE75292074C6
:1007BF001F552E700375290AD0F0D0E0D0D0C2D3C8
:1007CF00D2AF327901E1EA7903E1EA790AE1EA7914
:1007DF001EE1EA7964E1EA79C8E1EA7817E4D5E045
:1007EF00FDD8FAD9F6227A147B780208117A107B99
:1007FF008C0208117A0D7BB40208117A0B7BC802A8
:10080F000811AC257525017902B275E4C282D5E0D5
:10081F00FDE5256002D294D5E0FDC294D5E0FDD26E
:10082F0082D5E0FDE525600A207502D2833075027E
:10083F00D295E56DD5E0FD207502C283307502C2F9
:10084F00957496D5E0FDD9C1EAF8D5E0FDD8FBDB6C
:10085F00B1C2828C2522C37C007D0075F00005F0AB
:0F086F00EA33FAEB33FB50F6EB13FBEA13FAC351
:10087E00E9FFE8FEE89AF8E99BF95004EFF9EEF883
:10088E00B3EC33FCED33FDD5F0DFEDF9ECF822E8F7
:10089E0089F08A20D2D4F8A9F07B0030F70B7BFFC9
:1008AE00F42401F8E9F43400F9E88520F0A4ADF061
:1008BE00F8E98520F0A4AFF0FEED2EF974003FFAB2
:1008CE007C04C3EA13FAE913F9E813F8DCF48BF0AD
:1008DE0030F70AE8F42401F8E9F43400F9E889F075
:1008EE00C2D4F8A9F0227882B60403020980C3E5C7
:1008FE005894014018E54870377805C37994B702CB
:10090E00027812C3E53B9400E53C984020E5486030
:10091E0009855E5D7562FF756301852224E4F53FEE
:10092E00F540F541F542F543F54802098075480159
:10093E00C37994E79402601BE523F43333F913F87B
:10094E00E9540104F9E854FEC39440F8E99400F91F
:10095E0002097CE523F433333333F913F8E95407F2
:10096E000404F9E854F8C39440F8E99400F9883F78
:10097E00894022E548603BC3E53C13F9E53B13F89B
:10098E00C3E53F98F8E54099F9500CC3E89480E927
:10099E0094FF40160209BCC3E8947FE9940050030B
:1009AE000209BC787F79000209BC788079FF8844FF
:1009BE00894522E5486058E5442541F8E54535422C
:1009CE00F9854520E4300701F43543FA30E709C3D1
:1009DE00EA94F040150209FEC3EA940F500302098F
:1009EE00FE78FF79FF7A0F0209FE780079007AF01F
:1009FE00C3E524955C5006E52460094117E54520C2
:100A0E00E70D4117E54530E706884189428A4322C2
:100A1E00E5487003020A81789EE6FAC3E54433F88E
:100A2E00E54533F9119DE930E70BC3E89480E9946D
:100A3E00FF40134158C3E8947FE994005002415897
:100A4E00787F79004158788079FFE820E715C3E573
:100A5E002398F84009C3E894014003020A7F780105
:100A6E00020A7FE8F424012523F84003020A7F7866
:100A7E00FF884622E5487003020AE3789FE6FAA84B
:100A8E0042A943119DE930E70CC3E89401E994FFB4
:100A9E004016020ABAC3E894FFE994005003020A12
:100AAE00BA78FF7900020ABA780179FFE920E715D2
:100ABE00C3E54698F84009C3E894014003020AE1F1
:100ACE007800020AE1E8F424012546F84003020A00
:100ADE00E178FF8824227883E6F52012102175E84C
:100AEE0090E5E820ECF0A8BDA9BE1210B6756855C9
:100AFE00756900C3740013FD745513FC74552CFCFA
:100B0E0074003DFDECFAEDFBC3E89AE99B4014E559
:100B1E00682455F568E5693400F569EA2CFAEB3D71
:100B2E00FB80E5AE68AF69C3E56913F9E56813F8B4
:100B3E00C3E913F9E813F8E56828F566E56939F5B0
:100B4E00677A03C3E913F9E813F8DAF7AA201A70E3
:100B5E0009756800756900020B781AEA6008EE28BC
:100B6E00FEEF39FFDAF88E688F692275E8902278E9
:100B7E0083E6FFE5E820ECF7A8BDA9BE056AC3E54C
:100B8E006A94084052756A00E97007E56B601B02B3
:100B9E000BACC3E8956B6010E56B5006600C14024D
:100BAE000BB80460F9020BB8E56BF56BC3946DF8E6
:100BBE004021755CC0C3E89404F84017755C80C38F
:100BCE00E89404F8400D755C40C3E89404F84003C3
:100BDE00755C0075BB0922EFC39401601BC3E894DA
:100BEE00FFE994035012C3E89568E995695009E549
:100BFE005C600C155C020C0DE55CF46002055CA8F3
:100C0E005CC3E524985002A8248825C3E525955D8C
:100C1E00400B855D25E55DF46003855D5CC3E56A8B
:100C2E00B4070375BB10223061027832306202784D
:100C3E0050E52C5406601FE879A187F0A4C5F0A2F8
:100C4E00F733F8C3E8955C4002A85C8822882488B4
:100C5E0025306102885E22788FE6FFC3EF9405503F
:0F0C6E0018C3EF94045020C3EF94035028C3EF32
:100C7D0094025030C3EF940150387533A075340F82
:100C8D0075353C75360581CD7533C07534127535A6
:100C9D004075360681CD7533707534177535D07541
:100CAD00360781CD75334C75341D7535C4753609D0
:100CBD0081CD7533287534237535B875360B81CDD7
:100CCD0085334F853450753B00753C0822A84FA9DC
:100CDD0050020CE5A849A94A759100C3E498F59412
:100CED00E499F595759104D25875C820A8CCA9CD75
:100CFD0075C824AA39AB3A8839893AC3E89AF8E914
:100D0D009BF9AA3BAB3CC3EB13FDEA13FCC3ED13FC
:100D1D00FDEC13FCC3EA9CFAEB9DFBEA28FAEB39D8
:100D2D00FB8A3B8B3C400122753BFF753CFF22301B
:100D3D005802A13C759100C3E4954BF594E4954C94
:100D4D00F595759104D258227892E6FF7E10305BAE
:100D5D00027F053063047F037E00A93CA83B7A0423
:100D6D00C3E913F9E813F8DAF7C3E89EF8E994003C
:100D7D00F94009C3E89402E9940050047802E4F9BB
:100D8D00E9FBE8FAC3E913FDE813FCC3EF94036034
:100D9D002EEF20E00DE82CF8E93DF9ECFAEDFB0221
:100DAD000DB9E828F8E939F97A02E4FBC3EF9403A9
:100DBD00400D8A4D8B4E8849894A8C4B8D4C22882B
:100DCD004D894E8A498B4A8C4B8D4C22305802A14D
:100DDD00D9759100C3E4953BF594E4953CF5957573
:100DED009104D25822753E00752000020E01753E09
:100DFD0000752040D2AF053E20580122759D00E5BB
:100E0D003CC313C313F8086030306A06C313C31311
:100E1D00F808C3E8940A4002780A306D08C3E894D4
:100E2D000440027804C3E53C9408400D759D02C34F
:100E3D00E53C94104003759D03205803D2AF2279F1
:100E4D001E206D02790AD2AF0000C2AF205A0A7976
:100E5D003C206D027914306FE03063027978C3E580
:100E6D008B9920630240F740D0E59BF4F45440B5D4
:100E7D002002C101D8C3D2AF22C25B789CE61460B8
:100E8D0007E53E147002D25B30630B053820581015
:100E9D00753800020EAD205807158115810217F522
:100EAD0022759100C3E4954DF594E4954EF5957535
:100EBD009104D25822AE25305B4F78A3E6FFBF01D7
:100ECD000BD25C752500C283C294C295B141305CD2
:100EDD0003752500305802C1DBBF020BD25C7525AE
:100EED0000C283C294C29578A2B6010DB141305CA7
:100EFD0003752500305802C1FBBF030BD25C75256D
:100F0D0000C283C294C295D1AE305C03752500300A
:100F1D005802E116305B04C25C8E2522C2AFC2823C
:100F2D00206A03020F4890034B306E0F207502C2EA
:100F3D0097307502C2807406D5E0FD207502D2800F
:100F4D00307502D297759F43753D02D2AF22C2AF65
:100F5D00206A03020F7D900302306E17C282207546
:100F6D0002C297307502C2807406D5E0FD020F8073
:100F7D009001E5207502C295307502C283305A0684
:100F8D00E5256002D294207503759F533075037566
:100F9D009F33753D03D2AF22C2AF207502C28030A0
:100FAD007502C297206A03020FC49002C1306E070A
:100FBD00C2827406D5E0FD207502D297307502D23B
:100FCD0080207503759F33307503759F53753D04F0
:100FDD00D2AF22C2AF206A03021002900280306E9F
:100FED0017207502C280307502C297C2827406D571
:100FFD00E0FD0210059001D3C294305A0EE5256034
:10100D000A207502D283307502D295759F43753DC6
:10101D0005D2AF22C2AF207502C297307502C280D1
:10102D00206A03021048900237306E0F207502C2FD
:10103D0080307502C2977406D5E0FDD2822075030B
:10104D00759F53307503759F33753D06D2AF22C220
:10105D00AF206A030210869003A4306E1F20750224
:0F106D00C280307502C297207502C2973075029B
:10107C00C2807406D5E0FD0210899001F72075023C
:10108C00C283307502C295305A0EE525600A207570
:10109C0002D295307502D283207503759F3330755B
:1010AC0003759F53753D01D2AF229001D1C283C20B
:1010BC0094C295C280C282C29722C3E54F9535E592
:1010CC005095365001227890E6FFC3EF94055018E6
:1010DC00C3EF9404501BC3EF9403501EC3EF940250
:1010EC005021C3EF94015024C3E54F943CF80211F6
:1010FC0021C3E54F9428F8021121C3E54F941AF847
:10110C00021121C3E54F9412F8021121C3E54F944B
:10111C000AF8021121E5509400F9884F89502230C9
:10112C00580302112B227880760778817607788213
:10113C007601789476017883760478867609788FB0
:10114C007603789076017895760278927603789B80
:10115C00760D7893760178877602789C760178887C
:10116C0076017889760178857600788C7601788D91
:10117C007600788E76B478967625789776D07898AF
:10118C007678789976C8789A7604789D7600227865
:10119C0093E6FF756409756501C3BF0209756405A3
:1011AC007565010211E0C3BF03097564057565021D
:1011BC000211E0C3BF04097564057565030211E0F3
:1011CC00C3BF0506756409756507C3BF060675645C
:1011DC00007565007887E6FFC26CC3BF0302D26C52
:1011EC00C26BC26A7418552D6002D26AC26E60025C
:1011FC00D26ED26F6002C26FC2757888E630E1029F
:10120C00D275C2767889E630E102D276C3EF9402C9
:10121C006008758E01D26D02122B758E00C26D2284
:10122C007880E61490008093789EF67881E614908E
:10123C00008093789FF611B622789BE61490008D6F
:10124C009378A0F611B6227886E61490009A9378DB
:10125C00A1F611B622789CE6149000A79378A2F61A
:10126C00789CE6149000AC9378A3F611B622227801
:10127C0096E6FA7897E6FB3077047A007BFFC3EBAF
:10128C009AFCC3948250027C82756C00056CEC85D0
:10129C006CF0A4C3E5F0948040F222C2D353D9BFC2
:1012AC007581C043FF801207D275EF0243B203E58C
:1012BC00B324044002F5B37580F275A40D75F13FAB
:1012CC0075D4DF75904F75A5B075F2F075D50075B6
:1012DC00A60175E24111B6E4F8F6D8FD31321218C8
:1012EC0040319B512C514551535161517A517B786E
:1012FC0098866D11B675885075890275C8247591DC
:10130C000475D8401207E61207F51207DE1207FC27
:10131C001207DE1208031207DE121CE51207E61292
:10132C0007E61207E275A82275B80275E69075F605
:10133C0010759B80759D0375D10E75BC5875BB09D6
:10134C0075BA1175E8801207D2D2AF120AE443DAEB
:10135C0001C2D8C2691207E6753001D2597A05E587
:10136C005770027A051207D6E558C3940240EEE591
:10137C002E541F855A59F55AB559E2DAE2C259531F
:10138C00DACF20760343DA2030760343DA10C2D862
:10139C00C2691207E21207D67802741F552E70022A
:1013AC007800C3E5589840EDC2AF1207F51207F567
:1013BC001207F5D2AF1207E67547001207D6788CE4
:1013CC00E6C394015003021490E530C3940150031A
:1013DC00021490741F552E6035C3E55894FF5003CA
:1013EC00021490C2AF12080AD2AF1207E2C3E5583A
:1013FC00940150EFC2AF1207F51207DA1207F5D2BB
:10140C00AF1207E2C3E55894FF40E9021D6A7F055D
:10141C00D277517B1207E2C2AFC277517BC3E5583A
:10142C00947FD2AF4068C2AF12080AD2AFDFE1C3DB
:10143C00E55894057897F61207E61218F0121CED91
:10144C007F0AD277517B1207E2C2AFC277517BC3BE
:10145C00E558947FD2AF50E8C2AF1207F51207DA05
:0E146C001207F5D2AFDFDBE55824057896F6BF
:10147A001207E61218F0121D1C1207E2C3E558946F
:10148A00FF40F6021D6AC3E5589547400385584751
:10149A001207E2C3E5589401400261C7C2AF1208BD
:1014AA000A12080A12080AD2AF1207E6753000E4D7
:1014BA00F531F5320531E531F470360532789AE6C0
:1014CA007828146012785014600D78A01460087897
:1014DA00F0146003753200C3E5329840141532786F
:1014EA0099866DC2AF12080AD2AF7898866D120734
:1014FA00E21207D6E5287008741F552E700261673C
:10150A00C3E558940640AD1207E2E52870030213BA
:10151A006711B6E4F522F523F524F525755CFF7805
:10152A0085865FF53FF540F541F542F543F56AF5E5
:10153A0048F52BF52CF55B120C65756A0875BB101E
:10154A001207D2120B79E5E820ECFBA8BDA9BEE987
:10155A007001F8886B120B7D756A0875BB10789557
:10156A00E630E0030215AB7887E6FE7602319B7817
:10157A0087EEF6D261C2AF120C3585225C85225DF8
:10158A00D2AFC261752500756200756301D260D25F
:10159A00637538001121115C120CE1120C650216F8
:1015AA00CD7887E6FE76037893E6FD7605319B785B
:1015BA0087EEF67893EDF6D260D261D26E112111E0
:1015CA005C120C351207D2120F291207D21207D257
:1015DA00120F5B1207D6120FA51207D61207D612E0
:1015EA000FE01207DA11211207D61207D2C261D20E
:1015FA0062120B79120B7D120C35756A0875BB10D5
:10160A00115C120CDA120D5511C6312B120F291268
:10161A000CDA120D5511C6312B120F5B120CDA12AD
:10162A000D5511C6312B120FA5120CDA120D5511D8
:10163A00C6312B120FE0120CDA120D5511C6312BDE
:10164A001121120CDA120D5511C6C3E54F9535E575
:10165A00509536400C312BC3E5589401509302172C
:10166A00F5312BC2627887E6FE7602319B7887EEE7
:10167A00F685225C855E5D855E257562007563016F
:10168A00D263753800C2AF207502C280307502C2BB
:10169A0097207502C297307502C280742DD5E0FD7D
:1016AA00D2AF115C120CE1120D3C120D55120DD97C
:1016BA00756A0075BB090216CD319B115C756A000B
:1016CA0075BB09120DFB120E86120EAE1208F41229
:1016DA000EC2120F29120CE1120D3C120D55120DF9
:1016EA00D9120DF2120E86120EAE120981120EC214
:1016FA00120F5B120CE1120D3C120D55120DD9128C
:10170A000DFB120E86120EAE1209C1120EC2120F74
:10171A00A5120CE1120D3C120D55120DD9120DF243
:10172A00120E86120EAE120A1E120EC2120FE0120C
:10173A000CE1120D3C120D55120DD9120DFB120EB1
:10174A0086120EAE120A82120EC21121120CE11278
:10175A000D3C120D55120DD9120DF2120B79120E03
:10176A0086120EAE120B7D120EC2115C120CE11221
:10177A000D3C120D55120DD930632A855E5C855ECB
:10178A005D756200756301C3E5389464400AC263FB
:10179A00D2647537140217AFC3E5589401400302A7
:1017AA0016CD0217F5306419E537147005C26402C4
:1017BA0016C3F537C3E558940140030216CD021744
:1017CA00F5C3E55B94014009855E5D7562FF75634B
:1017DA0001C3E55B94FA5013741F552E7004E52873
:1017EA006009C3E53C94F05002C1CD11B67887E692
:1017FA00FE7602319B7887EEF6E4F522F523F5248E
:10180A00F525F55FC2601207D21210B6741F552E65
:10181A007007E52870030213677895E630E009122D
:10182A001CE5121CE5121CE5788DE6C39401400301
:10183A000213A10214B9901A0D7820121C00E52097
:10184A00B4A50CA3121C00E520B45A0302186212B4
:10185A0011321218F00218EF901A037880121C0045
:0F186A00A308121C00A308121C00A308121C00E4
:10187900A308A308A308121C00A308121C00A308AC
:10188900121C00A308121C00A308A308A308121C19
:1018990000A308121C00A308121C00A308121C00B4
:1018A900A308121C00A308A308121C00A308121CF9
:1018B90000A308121C00A308121C00A308121C0094
:1018C900A308121C00A308121C00A308121C00A3E1
:1018D90008121C00A308121C00A308121C00A3086C
:1018E900121C00901A2122C2AF121C3F121C19901F
:1018F9001A00740A121C05A37404121C05A374109F
:10190900121C05901A037880121C04A308121C04E7
:10191900A308121C04A308121C04A308A308A30803
:10192900121C04A308121C04A308121C04A3081205
:101939001C04A308A308A308121C04A308121C046E
:10194900A308121C04A308121C04A308121C04A354
:1019590008A308121C04A308121C04A308121C04DF
:10196900A308121C04A308121C04A308121C04A334
:1019790008121C04A308121C04A308121C04A308BF
:10198900121C04A308121C04A308121C04121C52E2
:07199900121C30901A2122FC
:101A00000A041007070104FFFF09020101A55A019A
:101A100000B40301FF0301010225D078C8040D01C1
:021A200000FFC5
:101A400023416C69676E424C333558232020202097
:101A500023424C48454C4923463333302320202031
:101A60002020202020202020202020202020202076
:101C0000E493F622E6438F01538FFD75EF0275B71B
:101C1000A575B7F1F0538FFE22438F02438F0175F4
:101C2000EF0275B7A575B7F1901A0DF0538FFC222E
:101C3000901A0D74A59105901A0E745A9105227A86
:101C40003079D07820901A409100E520F709A3DA86
:101C5000F7227A3079D0901A40E7910509A3DAF992
:101C600022AB6EA86FBB01057980021CE2BB0205A6
:101C70007981021CE2BB03057982021CE2BB0405E8
:101C80007994021CE2BB05057983021CE2BB0605C0
:101C90007995021CE2BB07057986021CE2BB0805A8
:101CA000798F021CE2BB09057990021CE2BB0A0590
:101CB0007992021CE2BB0B05799B021CE2BB0C056E
:101CC0007993021CE2BB0D057987021CE2BB0E056D
:101CD000799C021CE2BB0F057988021CE27989021B
:101CE0001CE2E8F7227C051207E6DCFB22C2AF12F9
:101CF00007F51207FC12080312080A1207DA120786
:101D0000F51207FC12080312080A1207DA1207F587
:101D10001207FC12080312080AD2AF22C2AF12083F
:101D20000A1208031207FC1207F51207DA12080A52
:101D30001208031207FC1207F51207DA12080A123A
:101D400008031207FC1207F5D2AF22AE6EAF6FC2C6
:101D5000AF1207F51207F51207F51207DADEF212D5
:101D6000080A1207DADFF8D2AF2291ED91E591E58A
:101D7000756E01756F01757000B14B7C05AD581221
:101D800007E6C3ED955870F5C3E55894014009C3C3
:101D9000E55894FF4032A1A691611218F091EDC26E
:101DA000AF75EF1291E5DCD50570C3E57094035073
:101DB0000280C691E5056FE56E149000B193F808B6
:101DC000C3E56F98500280AE91E591E5056EC3E5DD
:101DD0006E94115002809C1211321218F0C2AF752D
:041DE000EF1291E588
:00000001FF
